:020000020000FC
:1000000011C018951895189518951895B2C018959F
:100010001895A0C018951895189518957EC0189534
:100020001895189512E00FE51EBF0DBFA89508E1C1
:1000300001BD0EE101BDA895B0E0A0E615E009E024
:100040001D930A95E9F70FEF0ABB849900950BBB46
:1000500003E007BB002704BB0FEF05BB04E801BBAF
:1000600008E702BB01E006B90FEF07B901E001BFE5
:100070000BE003BF03E00EBD01E809BF002708BF86
:1000800001E009B900E000BD0EE800BD22270CB177
:100090002BB9579A549A7724172C552740E008E03B
:1000A000802E33B230944424A895789442FD01C048
:1000B000FDCF4B7F539409F46394213029F0223013
:1000C000D9F02330E0F4F2CF662329F5239541607F
:1000D000B0E0A0E66624552433B2309444242A9B31
:1000E00043943114410409F0E1CF18E000270D9347
:1000F0001A95E9F72227DACF53146404B9F61D9153
:10010000611719F0AA956D93406823952A3070F213
:1001100022274260CBCF2227C9CF3FB70F931F932F
:10012000550F09F451E018E0F0E0E0E622240191D7
:10013000052321F0220C1A95D1F704C00894221C43
:100140001A95A9F7849920942BBA51BF1F910F914A
:100150003FBF18953FB75C9906C05B9907C04460E4
:100160006CB13FBF189521E05C98FACF22275B98CD
:10017000F7CF3FB70F93A89547FD19C0389A7694EB
:1001800070FC02C0979A01C097988A9449F400279E
:1001900041FF0AE040FF02E0702E4C7F08E0802E15
:1001A00006EE0DBD08E70CBD0F913FBF18954F77C8
:0E01B000389B02C03898E3CF389AE1CFFFCFDA
:00000001FF
